:10000000850186018316FF3085008601831200304A
:100010009700970CAA309600851D112805199A2A79
:10002000BB2905190829960C0330161C04308F00D3
:1000300063308D0003308E00053090000530920053
:1000400005309400061017309100000000000000F9
:100050000614910B292800000000900B22280000B4
:10006000061016309300930B3328061402309500C7
:10007000950B38280000920B30280000061017302E
:1000800091000000000000000614910B45280000BC
:100090000000940B3E280000860D000000000000C8
:1000A00000000000000000001530061C1B3E8C0004
:1000B0000614161C5B28861000008C0B5D280000BF
:1000C000061002309500950B6328000000003030C8
:1000D0008C0006148C0B6A2800008F0B602800002F
:1000E000061002309500950B7328000000001F30A9
:1000F0008C000614000000000000053098009900F4
:100100009A009B009C009D009E009F001D30860071
:10011000980B882819308600990B8C28153086009A
:100120009A0B9028113086009B0B94280D30860086
:100130009C0B9828093086009D0B9C280530860072
:100140009E0BA028013086009F0BA4280000000011
:10015000000000008D0B7028000006100230950092
:10016000950BB02863308D001F308C000614000002
:10017000000000000530980099009A009B009C0048
:100180009D009E009F001D308600980BC5281930E9
:100190008600990BC928153086009A0BCD2811309E
:1001A00086009B0BD1280D3086009C0BD52809308A
:1001B00086009D0BD928053086009E0BDD28013076
:1001C00086009F0BE12800000000000000008E0B5D
:1001D00070280000061000000000003016180130E2
:1001E000970000000F301618183E8C000614161CDD
:1001F000F928000000008C0BFB28970C05190C282F
:1002000085190C28000000000000000000001328E1
:10021000960C0330161C04308F0063308D000330C1
:100220008E000530900005309200053094000610D5
:10023000173091000000000000000614910B1E29E9
:1002400000000000900B17290000061016309300E4
:10025000930B2829061402309500950B2D290000D8
:10026000920B2529000006101730910000000000B5
:1002700000000614910B3A2900000000940B33296A
:100280000000860D000000000000000000000000DB
:1002900000001530061C1B3E8C000614161C50294D
:1002A000861000008C0B52290000061002309500C9
:1002B000950B58290000000030308C0006148C0B80
:1002C0005F2900008F0B55290000061002309500B1
:1002D000950B6829000000002C308C0006140000EB
:1002E000000000000000000000000000000000000E
:1002F0001D3086008C0B7A29013086008D0B652914
:100300000000061002309500950B842963308D00A3
:100310002C308C00061400000000000000000000DB
:1003200000000000000000001D3086008C0B9629A4
:10033000013086008E0B65290000061000000000C9
:10034000003016180130970000000F301618183EC4
:100350008C000614161CAC29000000008C0BAE2982
:10036000970C051D0C2885190C28000000000000C2
:10037000000000000829960C0000000004308F00E7
:100380001C308D000A308E00043090000530920041
:1003900005309400061017309100000000000000A6
:1003A0000614910BD12900000000900BCA2900000F
:1003B000061016309300930BDB29061402309500CB
:1003C000950BE0290000920BD82900000610173089
:1003D00091000000000000000614910BED290000C0
:1003E0000000940BE629000000000000000000005F
:1003F00000000000000000001530000000008C002C
:100400000000000000000000861000008C0B062A8F
:100410000000061002309500950B0C2A0000000029
:1004200030308C0006148C0B132A00008F0B092A25
:100430000000061002309500950B1C2A00000000F9
:100440000930A000061400000000000000000000B9
:1004500000000000000000001C308607860200003B
:1004600002308C008C0B322AA00B2C2A00001C308E
:100470008607860200000000000000000000000067
:100480008D0B192A0000061002309500950B462AA4
:10049000000000002C308C0006140000000000005A
:1004A0000000000000000000000000001D30860079
:1004B0008C0B582A01308600000000000000061056
:1004C00002309500950B622A1C308D002C308C0078
:1004D0000614000000000000000000000000000002
:1004E000000000001D3086008C0B742A013086004D
:1004F0008E0B192A000006100000000000301618AC
:100500000130970000000F30000000008C0006143E
:10051000000000000000000000008C0B8D2A970CEA
:1005200005190C28851D0C280000000000000000A3
:100530000000BB29960C0000000004308F001C3026
:100540008D000A308E000430900005309200053096
:1005500094000610173091000000000000000614FF
:10056000910BB02A00000000900BA92A0000061091
:1005700016309300930BBA2A061402309500950B9F
:10058000BF2A0000920BB72A000006101730910016
:100590000000000000000614910BCC2A00000000AF
:1005A000940BC52A000000000000000000000000BD
:1005B0000000000000001530000000008C0000006A
:1005C000000000000000861000008C0BE52A0000EF
:1005D000061002309500950BEB2A00000000303029
:1005E0008C0006148C0BF22A00008F0BE82A000006
:1005F000061002309500950BFB2A000000003030F9
:100600008C0006148C0B022B00008D0BF82A0000C6
:10061000061002309500950B0B2B000000000930EE
:10062000A000061400000000000000000000000010
:100630000000000000001C30860786020000023027
:100640008C008C0B212BA00B1B2B00001C30860771
:100650008602000000000000000000000000000012
:1006600000000000061002309500950B352B1C3061
:100670008D000930A00006140000000000000000FA
:10068000000000000000000000001C308607860209
:10069000000002308C008C0B4B2BA00B452B000074
:1006A0001C308607860200000000000000000000E9
:1006B00000008E0BF82A0000061000000000003039
:1006C00016180130970000000F30000000008C0069
:1006D0000614000000000000000000008C0B6E2BD0
:1006E000970C051D0C28851D0C280000000000003B
:0606F000000000009A2A40
:00000001FF
